:0A2244000001020203030404050573
:100D0200E4F562F561F560F55FC209C206C208C288
:100D120007122147120B177E187F008E0A8F0B7560
:100D2200121875131275081875091C7510187511AB
:100D32005175141875157FEE54E07003020E497553
:100D420063007564808E658F66C374A99FFF7418F3
:100D52009ECF2402CF3400FEE48F5E8E5DF55CF5FB
:100D62005BF55AF559F558F557AF5EAE5DAD5CAC23
:100D72005BAB5AAA59A958A857C3120FA25026E52D
:100D820064255AF582E5633559F58374CDF0E55A49
:100D92002401F55AE43559F559E43558F558E43546
:100DA20057F55780C4E4F55AF559F558F557AF5E33
:100DB200AE5DAD5CAC5BAB5AAA59A958A857C31239
:100DC2000FA25031AE59AF5AE5662FF582E5653E66
:100DD200F583E0FDE5642FF582E5633EF583EDF0F2
:100DE200EF2401F55AE43EF559E43558F558E43557
:100DF20057F55780B985630A85640B74002480FF18
:100E0200741834FFFEC3E5139FF513E5129EF51225
:100E1200C3E50D9FF50DE50C9EF50CC3E50F9FF59F
:100E22000FE50E9EF50EC3E5099FF509E5089EF54F
:100E320008C3E5119FF511E5109EF510C3E5159F56
:100E4200F515E5149EF514D2E843D82090E668E043
:100E52004409F090E65CE0443DF0D2AFD288D28AF9
:100E6200C2A8C2AA43E808D2FB90E680E020E105CE
:100E7200D20A121F1B90E680E054F7F0538EF8C29C
:100E8200093007051206EDC2073009291216FE5075
:100E920024C20912207420061690E682E030E7048C
:100EA200E020E1EF90E682E030E604E020E0E412A8
:0A0EB2001F4A12227412135D80C75C
:1006ED0090E6B9E0700302079E14700302081B2404
:1006FD00FE700302089E24FB70030207981470031A
:10070D00020792146073146076240560030208FDDD
:10071D00122276400302090990E6BBE024FE602216
:10072D0014603324FD601114602224067048E50A1C
:10073D0090E6B3F0E50B8037E51290E6B3F0E513E4
:10074D00802DE50C90E6B3F0E50D8023E50E90E6E7
:10075D00B3F0E50F801990E6BAE0FF121F76AA06F6
:10076D00A9077B01EA494B600DEE90E6B3F0EF90DF
:10077D00E6B4F00209090209021221CD020909129B
:10078D002260020909121C910209091221BB0209FA
:10079D0009122278400302090990E6B8E0247F602F
:1007AD001514601924027063A206E43325E0FFA23C
:1007BD0008E4334F8041E490E740F0803F90E6BC81
:1007CD00E0547EFF7E00E0D394807C0040047D01E8
:1007DD0080027D00EC4EFEED4F2444F58274223EE6
:1007ED00F583E493FF3395E0FEEF24A1FFEE34E6AD
:1007FD008F82F583E0540190E740F0E4A3F090E69A
:10080D008AF090E68B7402F00209090209021222A5
:10081D007A400302090990E6B8E024FE601624022E
:10082D00600302090990E6BAE0B40105C2060209A7
:10083D000902090290E6BAE0705590E6BCE0547EDC
:10084D00FF7E00E0D394807C0040047D0180027D1A
:10085D0000EC4EFEED4F2444F58274223EF583E408
:10086D0093FF3395E0FEEF24A1FFEE34E68F82F582
:10087D0083E054FEF090E6BCE05480131313541F34
:10088D00FFE0540F2F90E683F0E04420F0806D8060
:10089D006412227C506690E6B8E024FE60192402B2
:1008AD00705A90E6BAE0B40104D206804F90E6BAD1
:1008BD00E064026047803E90E6BCE0547EFF7E001F
:1008CD00E0D394807C0040047D0180027D00EC4EDD
:1008DD00FEED4F2444F58274223EF583E493FF33FD
:1008ED0095E0FEEF24A1FFEE34E68F82F5838008BC
:1008FD00120080500790E6A0E04401F090E6A0E0E1
:03090D004480F033
:0109100022C4
:0300330002227036
:0422700053D8EF321E
:10214700758CE0758AC0E58954F04401F589758E70
:0821570003D28CD2A9D2AF2201
:03005B0002091186
:10091100C0E0C083C082C0D075D000C004C006C092
:0109210007CE
:10092200AF91530780EF64806003020B0853917FFD
:10093200300503020B06E54C64047070D3E53A946B
:10094200C8E53994005003020B060535E53525E06C
:100952002462F582E43428F583E539F0A3E53AF020
:10096200E53525E02460F582E43428F583E0FEA332
:10097200E0FFD394C8EE9400402FEF25E0FFEE3362
:10098200FEEF2444FFEE34FDFEE53525E02462F55A
:1009920082E43428F583E0FCA3E0D39FEC9E400977
:1009A200752B01754C00753500020B00E54C640196
:1009B2006003020A66D3E53A94C8E539940050030D
:1009C200020B060535E53525E02462F582E434287C
:1009D200F583E539F0A3E53AF0E53525E02460F545
:1009E20082E43428F583E0FEA3E0FFD394C8EE94BA
:1009F20000406EEF25E0FFEE33FEEF2444FFEE34BD
:100A0200FDFEE53525E02462F582E43428F583E035
:100A1200FCA3E0D39FEC9E4048054DE54D64027077
:100A22003DE53514F532752B01E53525E0245EF5FB
:100A320082E43428F583E0FEA3E024C8F537E43EDF
:100A4200F536E53525E02460F582E43428F583E0C7
:100A5200FEA3E024C8F543E43EF542754C0075352B
:100A620000020B00E54C64027061C3E53A94C8E5EC
:100A72003994004048D3E53A94C8E53994004010CF
:100A8200D3E53A9543E53995425005752B00802709
:100A9200D3E53A9543E5399542400FD3E53A953788
:100AA200E53995365004052B800DD3E53A9537E5A7
:100AB2003995364008052B753900753A00E52B65E6
:100AC2002C7041F54CF539F53A8039E54CB40534D2
:100AD200D3E53A9401E53994004029E53525E0242F
:100AE20062F582E43428F583E539F0A3E53AF005AE
:100AF20035052BE52BB41406754C00752B007539A2
:060B020000753A00C20577
:0F0B0800D007D006D004D0D0D082D083D0E03236
:101800001201000200000040181623160000010219
:1018100000010A0600020000004001000902350034
:1018200001010080FA0904000005FF00000007051F
:101830000102400000070582020002000705810244
:1018400040000007058602000200070508020002AA
:101850000009022E0001010080FA0904000004FFC3
:101860000000000705010240000007058202400059
:101870000007050202000200070581024000000483
:1018800003090410035100480059002D0043004390
:101890000044001603510048005900310036003260
:0B18A00000300030002000200000009D
:100495006080299C030A030302020307000000028F
:1004A500000002000A2B0B131115111100000000AA
:1004B5000000003F020A03030303030700000002D4
:1004C500000002000A2B130B11151111000000008A
:1004D5000000003F032D0303030303070000000290
:1004E500000002000A2B0B1311151111000000006A
:1004F5000000003F030A0A0A0A0A0A070000000270
:10050500000002000A2B130B111511110000000049
:100515000000003F60242A230000000000000000C6
:1005250000000000000000000000000000000000C6
:10053500000000000000000000000000472A1C80A9
:06054500000009CA4E008F
:1015450090E60174CAF090E6F574FFF0902A1CE06D
:1015550090E6F3F0902A1DE090E6C3F0902A1EE095
:1015650090E6C1F0902A1FE090E6C2F0902A21E0B3
:1015750090E6C0F0902A22E090E6F4F075AF07748B
:1015850029F59A749CF59B759DE4E4F59EFF90E61C
:101595007BE090E67CF00FBF80F490E67174FFF07D
:1015A500F5B490E672E04480F043B680000000E4B4
:1015B50090E6C4F000000090E6C5F0902A23E09084
:1015C500E6C6F0902A24E090E6C7F0902A25E09040
:1015D500E6C8F0902A26E090E6C9F0902A27E09028
:1015E500E6CAF0902A28E090E6CBF0902A29E09010
:0B15F500E6CCF0902A2AE090E6CDF052
:0116000022C7
:03004300021700A1
:0300530002170091
:1017000002215F000221A50002218F000221770043
:10171000021E1800021DA40002227E0002227F0089
:101720000222800002228100021EEA000219450006
:1017300002228200022283000217B800021CF0007D
:101740000222840002227F000222850002228600FB
:1017500002228700022288000222890002228A00D7
:1017600002228B0002227F0002227F0002227F00E1
:1017700002228C0002228D0002228E0002228F00A3
:101780000222900002229100022292000222930083
:101790000222940002229500022296000222970063
:1017A000022298000222990002229A0002229B0043
:0817B00002229C0002229D00B0
:101F4A0090E682E030E004E020E60B90E682E030A2
:101F5A00E119E030E71590E680E04401F07F147E55
:0C1F6A00001216B390E680E054FEF02256
:1020740090E682E044C0F090E681F04387010000DE
:042084000000002236
:101F1B00300A0990E680E0440AF0800790E680E002
:101F2B004408F07FDC7E051216B390E65D74FFF07B
:0F1F3B0090E65FF05391EF90E680E054F7F022CC
:021F7600A907B9
:101F7800AE14AF158F828E83A3E064037017AD0192
:101F880019ED7001228F828E83E07C002FFDEC3EDC
:091F9800FEAF0580DF7E007F0032
:011FA100221D
:1016B3008E6B8F6C90E600E054187012E56C240179
:1016C300FFE4356BC313F56BEF13F56C801590E6F0
:1016D30000E05418FFBF100BE56C25E0F56CE56BDB
:1016E30033F56BE56C156CAE6B7002156B4E6005D4
:0616F30012208880EE22A7
:102088007400F58690FDA57C05A3E582458370F96B
:012098002225
:10054B0060A528F518244242424242424224181028
:10055B007010101010101010107C3C42424204041A
:10056B00081020427E3C42420418040202424438E6
:10057B00040C14242444447E04041E7E4040405842
:10058B006402024244381C244040586442424224D4
:10059B00187E444408081010101010103C424242C0
:1005AB002418244242423C1824424242261A020298
:1005BB00243800000000007F000000000038448257
:1005CB0082828282B2CA4C38E7424242427E424227
:1005DB004242E7EE44442828101010101038101037
:1005EB00182828243C444242E7C18142299A000042
:1005FB004228E200004228E4000041280000412884
:10060B0001004128EB0002301040C104C103014836
:10061B00000125004428F1000000004428E70000F9
:10062B0000004128E6006080286200000000000006
:10063B0000000000000000000000000000000000AF
:10064B00000000000000000000000000000000009F
:10065B00000000000000000000000000000000008F
:10066B00000000000000000000000000000000007F
:10067B00000000000000000000000000000000006F
:10068B00000000000000000000000000000000005F
:10069B00000000000000000000000000000000004F
:1006AB0000000000000000000000013500014C01BB
:1006BB00012CFF012B0002390000013200014D001B
:1006CB000236000002420000014B00025300000200
:1006DB00332710012A05C185013D00013B00012F85
:0106EB00000E
:101FA2008F679028427403F0E4A3F07A287B427D85
:101FB200027F411221109028427401F0A3E567F0DC
:0B1FC2007A287B427D027F4102211043
:0B222E00C2B6C2B48FB1D2B4D2B62247
:0B223900D2B6C2B48FB1D2B4D2B6222C
:04212C00AE05AD0748
:10213000E4FCE4FBAF05122239AF061222390BBBD7
:0621400060F20CBC40EC53
:012146002276
:101FF800AE05AD077F1512222EAF0612222E7F5F87
:1020080012222E7F7512222EAF0512222E7F3F122A
:0A201800222E7F2512223902223900
:041A63007D017F3052
:021A6700AE03CC
:101A6900EDC454F0F567EE75F008A4F568BF2D04D0
:101A79007A0A8020BF51047A0B8019BF48047A0C76
:101A89008012BF59047A0D800BBF41047A0E80047D
:101A9900EF24D0FAE4FBEA75F00BA424F5F582E40F
:101AA9003428F583E5822BF582E43583F583E0F963
:101AB900E4FCE930E70DE56724032BFFE5682CFD1D
:0F1AC900121FF8E925E0F90CBC08E70BBB0BC7AF
:011AD80022EB
:10209900C2B77FC87E00121C7AD2B77FAE12222E39
:0F20A9007FA012222E7F7212222E7FAF02222ED4
:1018AB00122099E4FDFF12212C7B027D017F511246
:1018BB001A677B037D017F48121A677B047D017FCA
:1018CB0059121A677B057D017F31121A677B067DE2
:1018DB00017F36121A677B077D017F32121A677BF5
:1018EB0008121A637B09121A637B0A7D017F41126E
:1018FB001A677B027D027F31121A677B037D027FA1
:10190B0037121A677B047D027F2D121A677B057DC8
:10191B00027F30121A677B067D027F35121A677BB6
:10192B00077D027F2D121A677B087D027F30121A0A
:0A193B00677B097D027F32021A6704
:100B170090E600E054E74410F00000000000009069
:100B2700E61074A0F000000090E60B7401F090E668
:100B37001274E0F0000000E490E613F0000000906B
:100B4700E61474E2F000000090E61574A0F00000CF
:100B57000090E6D27402F090E6047480F000000082
:100B67007402F00000007406F00000007408F00042
:100B77000000E4F000000012154590E6187408F034
:100B870000000090E619F000000090E61AF000005F
:100B97000090E61BF0000000E490E671F075B47F6A
:100BA70075A07F90E672F075B6FF75B1FF90E6709D
:100BB700F075B2FF75B5FFC28CD2B01216F990E688
:100BC7001074A0F000000090E611F000000090E61D
:100BD7005EE04408F0000000E490E68DF0000000BD
:100BE70090E65EE04404F0000000E490E7C0F09077
:100BF700E7C4F0A3F0A3F0A3F090E7F0F090E68F3E
:100C07007440F000000090E65EE04440F000000011
:100C17007E027F0090F800E4F0A3DFFCDEFA90E6A6
:100C2700987402F0000000E490E699F00000007E5E
:100C3700027F0090F800E4F0A3DFFCDEFA90E65EA6
:100C4700E04480F0000000E490E69CF00000009093
:100C5700E69DF00000007F9AFE1217F775270075D2
:100C670028B4754E01754F907530107531B87551B0
:100C77000675522C12226890E67AE054FEF0E4FDE5
:100C87007F901221DF7F647E001216B37DFF7F42C3
:100C97001221DF7F647E001216B37D827F4E122100
:100CA700DF753CFF43A020E4F54090E782E53CF088
:100CB70090E781E540F01216F9D205754C017533BE
:100CC70027753410752A05121B4C7F887E13121C5A
:100CD7007A121B4C7F887E13121C7A7FB87E0B1208
:100CE7001C7A122099D2F9C2F8E4F54890E7C0E5DA
:0B0CF70048F043A01053917F0218AB9F
:0E221300EF2401FBE43EFA7D047F480220F434
:10202200E540C313FFC374809F90299BF0E49400A2
:1020320090299AF0E540D394004006753CFF43A0F6
:0920420020E540700353A0DF22E9
:10146000E4FC9028EDE0FEA3E02400FDEC3EFC90BF
:101470002800E0FEA3E07A002400FFEA3EFEC3ED70
:101480009FFFEC9EFE9028E2F0A3EFF09028E5E0AD
:101490002FF09028E4E03EF0D3EF9450EE64809477
:1014A0008050129028E2E0FAA3E0FBC394B0EA6413
:1014B00080947F501C9028E3E025E0FE9028E2E035
:1014C0003390299AF0A3CEF0E49028E4F0A3F080C2
:1014D000337C007D14AF03AE02120F0BAC06AD07D8
:1014E0009028E4E0FEA3E07802C333CE33CED8F9EF
:1014F0002DFFEC3EFE7C007D0A120F1D90299AEE16
:10150000F0A3EFF0D390299BE094FF90299AE06438
:101510008094804006E4F0A374FFF0C390299AE021
:10152000648094805004E4F0A3F090299AE0FEA334
:10153000E0FF7C007D02120F1DC3747F9FF0E49ECC
:0415400090299AF064
:011544002284
:101BBE007E287FEC1222139028EDE090E7C1F09082
:101BCE0028EEE090E7C2F090299BE090E7C3F090FA
:101BDE0028EBE0600B43A020753CFF1214608003DD
:101BEE00122022902842E53CF07A287B427D017F2C
:101BFE00211221109028427402F0A37480F07A28EA
:101C0E007B427D027F28122110E4902842F0902919
:101C1E009BE0902843F07A287B427D027F280221A8
:011C2E0010A5
:10135D000554E55470020553054BB53410E553B5EE
:10136D00330B121BBEE4F553F5541220D790E7C88A
:10137D00E54CF0A3E52BF0E54B652A7023E54C60B9
:10138D001414600C14600924FD600504700F8000B6
:10139D001222038008E4FF121FA253A0EFE4F54BC5
:1013AD0020000302145F75480190E7C0E548F0E5A1
:1013BD00A030E7032004F87FAE12222E90F00074C7
:1013CD00AAF0A37411F0A374CCF0A374EEF0E49022
:1013DD00E690F090E6917405F012102790F00074ED
:1013ED00AAF0A37411F0A374CCF0A374EEF0E49002
:1013FD00E690F090E6917405F07FAF12222EC200B8
:10140D00E4F54890E7C0E548F09028E6E064017007
:10141D002653A0F043A0047FD07E07121C7A53A060
:10142D00F043A00C7FD07E07121C7A53A0F043A08E
:10143D00087FD07E078018121B4C7FB87E0B121CC4
:10144D007A121B4C7F887E13121C7A7F887E1312B2
:03145D001C7A22D4
:0216FE00D322F5
:02227400D32273
:02227600D32271
:101C910090E680E030E73A00000090E6207402F020
:101CA100000000E490E621F000000090E6247402B8
:101CB100F0000000E490E625F000000090E62674B4
:101CC10002F0000000E490E627F0000000D201805D
:101CD10016000000E490E620F000000090E6217478
:0F1CE10040F0000000C20190E6BAE0F549D322BE
:1021BB0090E740E549F0E490E68AF090E68B04F076
:0221CB00D3221D
:0822600090E6BAE0F526D32256
:1021CD0090E740E526F0E490E68AF090E68B04F087
:0221DD00D3220B
:02227800D3226F
:02227A00D3226D
:02227C00D3226B
:10008000E4FFF56790E6B9E0244B605F147003026B
:10009000029324FA70030202CB24FA700302032FA6
:1000A00024F8700302037724FA70030203B9241DB5
:1000B0006003020491E490E68AF090E68BF090E60B
:1000C000A0E020E1F990E68BE0E4F5B390E601745E
:1000D000CAF0D20000000090E6047480F000000036
:1000E0007402F0000000E4F0020493E490E68AF069
:1000F00090E68BF090E6A0E020E1F990E68BE0D36B
:10010000943F4024E4F56774402567F582E434E7C2
:10011000F583E0FF74022567F582E43428F583EF68
:10012000F00567E567B440DF7F8A7E001217F7901D
:100130002802E0FF7E0012224E902803E075F004B2
:10014000A4FFAEF0122257902807E0C39402501388
:10015000902823E090E6C07005744EF08016749CE1
:10016000F08011902823E090E6C07005749FF08025
:1001700003749DF0902825E0F541902822E0F53F9A
:10018000902826E0F54A902830E0F53EA3E0FEA353
:10019000E07C002400F524EC3EF523902835E09027
:1001A00028E6F0902808E0F538E538700375380146
:1001B00090280DE0FEA3E07C002400F528EC3EF53D
:1001C00027A3E0FEA3E02400F54FEC3EF54E902877
:1001D00009E0FEA3E02400F531EC3EF530A3E0FE9B
:1001E000A3E02400F552EC3EF55190283DE0FFE4F9
:1001F000FDFEFBFAF97801120F53A804A905AA061F
:10020000AB07902813E0FEA3E07C002400FFEC3E47
:10021000FEE4FDEB2FFFEA3EFEED39FDEC38FCC0BD
:1002200004C005C006C00790283EE0FFE4FCFDFEC8
:10023000FBFA7901F8120F53D003D002D001D0009D
:10024000EF2BF547EE3AF546ED39F545EC38F54438
:10025000902811E0FEA3E07C002400F52EEC3EF592
:100260002DE4FD7F901221DF902803E0FCA3E0FD48
:10027000A3E0FEA3E0FF9028F1120FC69028F1A39F
:10028000E0FDA3E0FEA3E0FFE4FC9028F1120FC61E
:10029000020493E4F56774022567F582E43428F5D7
:1002A00083E0FF74402567F582E434E7F583EFF0DF
:1002B0000567E567B440DF000000E490E68AF000DF
:1002C000000090E68B7440F0020493E490E68AF01C
:1002D00090E68BF090E6A0E020E1F990E6BDE0909A
:1002E0002842F090E6BCE0902843F0E4F56790E601
:1002F000BEE0FFE567C39F501E74402567F582E4AA
:1003000034E7F583E0FF74442567F582E43428F58B
:1003100083EFF0056780D790E6BAE0C313FF90E65D
:10032000BEE02402FD7A287B421221100204939041
:10033000E7407415F0A37402F0A3740CF0A37426C4
:10034000F0A37407F0A374EEF0A37401F0A3740398
:10035000F0A37453F0300105E4A3F0800690E74960
:1003600074FFF0000000E490E68AF000000090E6E0
:100370008B740AF002049390E6BCE0902A47F07A6E
:100380002A7B477D017F501221107A2A7B477D010D
:100390007F5012211090E6BEE0FD7AE77B407F504F
:1003A0001220F4E490E68AF000000090E6BEE090AF
:1003B000E68BF0000000020493E490E68AF090E6F9
:1003C0008BF090E6A0E020E1F990E68BE0F567C2C3
:1003D0009890E740E0C394304014E532242FFFE4C6
:1003E00033FEE0D39FEE6480F8748098401190E76C
:1003F00040E0F4600302047EE54C600302047E43A7
:10040000A01090E740E0F4600AE0B4300DE52B6402
:10041000016007D205754C04807990E740E0C394F1
:10042000314070E532242FFFE433FEE0D39FEE64C9
:1004300080F8748098505CE024D1F52C652B6053D3
:10044000E0B40A03752C6190E740E0B40B03752C0F
:100450006290E740E0B40C03752C6390E740E0B491
:100460000D03752C6490E740E0B40E03752C659085
:10047000E740E0B40F03752C66754C02801590E7D9
:1004800040E0B4200EE54C700A43A010754C058086
:0404900002D322C3AE
:010494002245
:10215F00C0E0C083C082D2075391EF90E65D740157
:08216F00F0D082D083D0E032F1
:10218F00C0E0C083C0825391EF90E65D7404F0D03D
:06219F0082D083D0E03283
:1021A500C0E0C083C0825391EF90E65D7402F0D029
:0621B50082D083D0E0326D
:101E1800C0E0C083C08285100C85110D850D8285B8
:101E28000C83A37402F085080E85090F850F82853F
:101E38000E83A37407F05391EF90E65D7410F0D011
:061E480082D083D0E032DD
:10217700C0E0C083C082D2095391EF90E65D740836
:08218700F0D082D083D0E032D9
:101DA400C0E0C083C08290E680E030E72085080C64
:101DB40085090D850D82850C83A37402F085100EB0
:101DC40085110F850F82850E83A37407F05391EF5D
:0D1DD40090E65D7420F0D082D083D0E03224
:01227E00322D
:01227F00322C
:01228000322B
:01228100322A
:101EEA00C0E0C083C08290E65EE054FBF0000000D0
:101EFA0090E68F7440F00000005391EF90E65FE0A7
:101F0A004404F090E65EE04404F0D082D083D0E04E
:011F1A003294
:0D194500C0E0C083C082C0D075D000C007D4
:1019520090E65EE054F7F090E6A1E020E1F990E72E
:1019620080E01460121460222404603614603D1476
:10197200703F752200803A90E782E0F53C90E78163
:10198200E0F5409028EBE4F0802790E782E0902891
:1019920000F090E781E0902801F09028EB7401F0CC
:1019A200800F90E781E024FF92048005752200D227
:1019B2000200000090E68DE4F05391EF90E65FE0C4
:0A19C2004408F090E65EE04408F0EF
:0B19CC00D007D0D0D082D083D0E03212
:012282003229
:012283003228
:1017B800C0E0C083C08290E65EE054BFF000000045
:1017C80090E6987402F000000090E699E4F00000BA
:1017D8000090F800F0A3F05391EF90E65FE04440EA
:0F17E800F090E65EE04440F0D082D083D0E03253
:0F1CF000C0E0C083C082C0D075D000C004C00661
:101CFF0090E65EE0547FF090E6A6E020E1F990E6F2
:101D0F009CE0FE90E69DE07C002400F556EC3EF54D
:101D1F005500000090E69CE4F090E69DF05391EFA3
:0E1D2F0090E65FE04480F090E65EE04480F0D5
:0D1D3D00D006D004D0D0D082D083D0E032C8
:012284003227
:012285003226
:012286003225
:012287003224
:012288003223
:012289003222
:01228A003221
:01228B003220
:01228C00321F
:01228D00321E
:01228E00321D
:01228F00321C
:01229000321B
:01229100321A
:012292003219
:012293003218
:012294003217
:012295003216
:012296003215
:012297003214
:012298003213
:012299003212
:01229A003211
:01229B003210
:01229C00320F
:01229D00320E
:061601008F688C698D6A00
:1016070053680753B0F77F0A7E00121C7AE4F56B24
:10161700C37402956BFFE568A807088002C313D857
:10162700FC30E00543800280035380FD7F0A7E0083
:10163700121C7A4380017F0A7E00121C7A5380FEB7
:101647007F0A7E00121C7A056BE56BC3940340C0CA
:10165700E4F56BC37409956BFFE56AAE69A80708E3
:101667008005CEC313CE13D8F930E005438002803E
:10167700035380FD7F0A7E00121C7A4380017F0A94
:101687007E00121C7A5380FE7F0A7E00121C7A05A8
:101697006BE56BC3940A40BB43B0087F0A7E001218
:0C16A7001C7A53B0F77F0A7E00021C7A08
:0917F700AD07AC06E4FF02160187
:09224E00AD07AC067F0402160185
:09225700AD07AC067F010216017F
:1021DF00902842EDF0EFC313FF7A287B427D010276
:0221EF002110BD
:101C2F0053A0F043A0087FC47E09121C7A53A0F082
:101C3F0043A00C7FC47E09121C7A53A0F043A0046A
:101C4F007FC47E09121C7A53A0F043A0067FC47E86
:101C5F0009121C7A53A0F043A0027FC47E09121C04
:0B1C6F007A53A0F043A0037FC47E095D
:101C7A00EF7803C333CE33CED8F9FFEF4E6007EFC8
:071C8A001F70F81E80F52217
:0516F900D283D284221F
:1020D700C2837F027E00121C7AC284D2837F027E73
:0D20E70000121C7AD2847F027E00021C7A57
:1021F100E4FDFC1220D70DBD00010CBC0EF5BD7431
:01220100F2EA
:0122020022B9
:101147009028F1E0FCA3E0FDA3E0FEA3E0FF9028D8
:10115700E7120FC6E53FB40102C2B09028E6E0707F
:10116700061220B843A040E54160030212387522F9
:1011770001E47FE87E03FDFC9028E7E0F8A3E0F9AF
:10118700A3E0FAA3E0FBC3120FA25003021226E565
:1011970022640160030212267FDD7E031216B3125A
:1011A7001BBE9028E7E0FCA3E0FDA3E0FEA3E0243C
:1011B70018FFEE34FCFEED34FFFDEC34FFFC902805
:1011C700E7120FC69028E7E0FCA3A3A3E4FFFEFD08
:1011D700EC7818120FB390E7C4EFF09028E7A3E07C
:1011E700FDA3A3E4FFFEE4FC7810120FB390E7C55C
:1011F700EFF09028E7A3A3E0FEA3E4FFE4FDFC786B
:1012070008120FB390E7C6EFF09028E7E0FCA3E0E1
:10121700FDA3E0FEA3E0FF90E7C7EFF0021178E53A
:1012270022B401169028E9E0FEA3E0FF1216B3806E
:1012370009752201E522640160FA9028E6E070064C
:0E12470053A0BF122221E53FB40102D2B02213
:101AD9008F6E8E6D8D6C8C6BE4FFFEFDFCAB6EAA78
:101AE9006DA96CA86BD3120FA24057000000E4FF48
:101AF900FEFDE56BFC7818120FB390E6CEEFF0000F
:101B09000000E4FFFEE56CFDE4FC7810120FB390D1
:101B1900E6CFEFF0000000E4FFE56DFEE4FDFC78A0
:101B290008120FB390E6D0EFF0000000E56EFF90C9
:101B3900E6D1EFF000000075BB04000000E5BB3002
:031B4900E7FB2295
:081DE1008C6B8D6CAB07AA06A8
:101DE900E4FDFCC3ED956CEC956B5022EA90E6D0CE
:101DF900F0000000EB90E6D1F000000075BB050093
:0E1E09000000E5BB30E7FB0DBD00010C80D5ED
:011E170022A8
:10204B00AD07AC06000000ED25E0EC3390E6D0F0D8
:10205B00000000ED25E090E6D1F000000075BB0418
:09206B00000000E5BB30E7FB2298
:10102700C20253A0F043A0047FD07E07121C7A535C
:10103700A0F043A00C7FD07E07121C7A53A0F04388
:10104700A0087FD07E07121C7A9028E6E064017022
:101057002A53A0BF53A0F043A0047FD07E07121CE1
:101067007A53A0F043A00C7FD07E07121C7A53A0BE
:10107700F043A0087FD07E07121C7A1221F1754831
:101087000290E7C0E548F012114775480390E7C0A2
:10109700E548F0300203021146E4F569F56AC3E555
:1010A7006A9528E5699527500D1220D7056AE56AE4
:1010B70070EC056980E8E53ED39400400CE53EFD01
:1010C7007C00AF31AE30121DE1D3E5249400E52357
:1010D70094004007AF24AE2312204BE4F567F56870
:1010E700C3E5689552E5679551502C121FCDE4F57D
:1010F70069F56AC3E56A95387480F8656998500D93
:101107001220D7056AE56A70EA056980E60568E591
:101117006870CD056780C9E4F569F56AC3E56A9526
:101127004FE569954E500D1220D7056AE56A70ECB8
:0F113700056980E8AF47AE46AD45AC44121AD902
:011146002286
:101FCD00000000E53125E0E5303390E6D0F000006B
:101FDD0000E53125E090E6D1F000000075BB04006E
:0B1FED000000E5BB20E7033002F822F3
:101B4C0053A0F043A0097F287E0A121C7A53A0F000
:101B5C0043A0017F287E0A121C7A53A0F043A003F5
:101B6C007F287E0A121C7A53A0F043A0027F287EA5
:101B7C000A121C7A53A0F043A0067F287E0A121C7E
:101B8C007A53A0F043A0047F287E0A121C7A53A03B
:101B9C00F043A00C7F287E0A121C7A53A0F043A0BD
:101BAC00087F287E0A121C7AE4F52590E7CBE52500
:021BBC00F02215
:0D222100121C2F75250390E7CBE525F02258
:1020B800121C2F53A0F043A001121C7653A0F0432A
:0F20C800A009121C7675250190E7CBE525F022C3
:101D4A00052FE52FB40803E4F52FE52F70047F086B
:101D5A00803DE52FB401047F0A8034E52FB40204E4
:101D6A007F02802BE52FB403047F038022E52FB482
:101D7A0004047F018019E52FB405047F058010E56E
:101D8A002FB406047F048007E52FB4070C7F0C12DA
:0A1D9A001FA27F2D7E00121C7A228A
:10220300E54C600B053AE53A70020539121D4A2286
:08226800E4F51BD2E9D2AF221C
:101E4E0090E678E020E6F9C2E990E678E04480F08A
:101E5E00EF25E090E679F090E678E030E0F990E654
:101E6E0078E04440F090E678E020E6F990E678E0FD
:061E7E0030E1D6D2E9229A
:101EB800A90790E678E020E6F9E51B702390E6781C
:101EC800E04480F0E925E090E679F08D16AF03A9AB
:101ED800077517018A188919E4F51A751B01D322A9
:021EE800C32213
:101E8400A90790E678E020E6F9E51B702590E6784E
:101E9400E04480F0E925E0440190E679F08D16AF46
:101EA40003A9077517018A188919E4F51A751B0324
:041EB400D322C32250
:03004B0002125549
:10125500C0E0C083C082C085C084C086758600C0DA
:10126500D075D000C000C001C002C003C006C007D1
:1012750090E678E030E206751B0602133F90E678AB
:10128500E020E10CE51B64026006751B0702133FB5
:10129500E51B24FE605F14603624FE7003021330E4
:1012A50024FC700302133C2408600302133FAB17B0
:1012B500AA18A919AF1A051A8F82758300120EBCD8
:1012C50090E679F0E51A65167070751B05806B90D0
:1012D500E679E0AB17AA18A919AE1A8E82758300B4
:1012E500120EE9751B02E5166401704E90E678E072
:1012F5004420F08045E51624FEB51A0790E678E00F
:101305004420F0E51614B51A0A90E678E04440F05A
:10131500751B0090E679E0AB17AA18A919AE1A8ECD
:1013250082758300120EE9051A800F90E678E04475
:1013350040F0751B008003751B005391DFD007D06B
:1013450006D003D002D001D000D0D0D086D084D032
:0813550085D082D083D0E03284
:1020F400121E84E51B24FA600E146006240770F394
:0C210400D322E4F51BD322E4F51BD32208
:10211000121EB8E51B24FA600E146006240770F343
:0C212000D322E4F51BD322E4F51BD322EC
:030000000219D70B
:0C19D700787FE4F6D8FD75816E021A1EC0
:100EBC00BB010CE58229F582E5833AF583E02250EB
:100ECC0006E92582F8E622BBFE06E92582F8E22235
:0D0EDC00E58229F582E5833AF583E493224F
:100EE900F8BB010DE58229F582E5833AF583E8F03F
:100EF900225006E92582C8F622BBFE05E92582C8EB
:020F0900F222D2
:100F0B00EF8DF0A4A8F0CF8CF0A428CE8DF0A42EFA
:020F1B00FE22B4
:100F1D00C2D5EC30E709B2D5E4C39DFDE49CFCEEEF
:100F2D0030E715B2D5E4C39FFFE49EFE120FD2C386
:100F3D00E49DFDE49CFC8003120FD230D507C3E481
:060F4D009FFFE49EFE225E
:100F5300E88FF0A4CC8BF0A42CFCE98EF0A42CFC3D
:100F63008AF0EDA42CFCEA8EF0A4CDA8F08BF0A4BB
:100F73002DCC3825F0FDE98FF0A42CCD35F0FCEB1A
:100F83008EF0A4FEA9F0EB8FF0A4CFC5F02ECD39DF
:0F0F9300FEE43CFCEAA42DCE35F0FDE43CFC224C
:100FA200EB9FF5F0EA9E42F0E99D42F0E89C45F0A5
:010FB200221C
:100FB300E8600FECC313FCED13FDEE13FEEF13FF1C
:030FC300D8F12240
:0C0FC600ECF0A3EDF0A3EEF0A3EFF0229E
:1019E300020D02E493A3F8E493A34003F68001F20B
:1019F30008DFF48029E493A3F85407240CC8C33305
:101A0300C4540F4420C8834004F456800146F6DFD3
:101A1300E4800B0102040810204080900495E47ECA
:101A2300019360BCA3FF543F30E509541FFEE493C8
:101A3300A360010ECF54C025E060A840B8E493A38F
:101A4300FAE493A3F8E493A3C8C582C8CAC583CABA
:101A5300F0A3C8C582C8CAC583CADFE9DEE780BE72
:0106EC00000D
:100FD200BC000BBE0029EF8DF084FFADF022E4CC03
:100FE200F875F008EF2FFFEE33FEEC33FCEE9DECCC
:100FF200984005FCEE9DFE0FD5F0E9E4CEFD22ED12
:10100200F8F5F0EE8420D21CFEADF075F008EF2F5B
:10101200FFED33FD4007985006D5F0F222C398FD4C
:051022000FD5F0EA22E9
:00000001FF
